:100000009F01831691010730831299003F308316B8
:1000100085003F30870008308312A3006F148316D9
:10002000871607168312960116179616161597014E
:10003000971717171716971191019115A701A4018A
:100040000730930092016F11EF108C1E25281718AE
:10005000EF141408A500EF1C392823082502031DFE
:10006000362897115A30A6006F1537289715A70123
:10007000EC2800308A0027083E3E82004228D9281A
:10008000E028E72800308A00250EB600B60C360CB2
:1000900003394B3E82004F28D828D828A6280030A4
:1000A0008A00250CB600B60C360C0739583E820083
:1000B0006028A5288B288C288D288D28982898289A
:1000C00000308A0007302505663E82006E287228BF
:1000D00078287C28822886288A288A283A21A6001F
:1000E0006F158A288A30A6006F150130A7008A286C
:1000F0006921A6006F158A280230A7008B30A60060
:100100006F158A281321A6006F158A280330A700CF
:10011000A6016F15A528A528A5283A21A6006F15C8
:10012000F0302605B6000F30250536045121A528EC
:100130003A21A6006F150F302605B6000F302505B1
:10014000B700B70EF03936045121D82800308A00A4
:10015000250CB600B60C360C0739AF3E8200D82805
:10016000D828D828D828D828D828D828B728003080
:100170008A0007302505BD3E8200D828D828D82817
:10018000D828C528C628D128D528D8286F15A60173
:10019000133024020318D0282408F220A600A40A51
:1001A000D828A401A6016F15D828A6016F159715A8
:1001B000EC28250851213A21A6006F15A701EC284B
:1001C000250884218C30A6006F15A701EC2825088E
:1001D0002821A6016F15A7016F1DF1282608D0213F
:1001E000B1212328840001308A000408003E8200E7
:1001F00000000000000000000000000000000000FF
:1002000010340034083401340334053449344F3495
:1002100038342D34413407344734723461346D340A
:1002200073346F346E34A801831611182814911892
:10023000A814111928159119A815111A2816911A20
:10024000A816111B2817911BA8178312280808004D
:10025000A90029181114A918911429191115A919FF
:100260009115291A1116A91A9116291B1117A91BE4
:10027000911700340508AA000708AB00AC012A1842
:100280002C142A1AAC14AA182C152A19AC152B18E0
:100290002C16AB18AC162B192C17AB19AC172C0855
:1002A0000800AF00AD01AE012F182D14AF182D16A8
:1002B0002F19AD14AF192D152F1A2E14AF1AAE1415
:1002C0002F1B2E15AF1BAE152D0885002E0887009D
:1002D0000034B201831605088312B00083160708A4
:1002E0008312B10030183214301AB214B01832151B
:1002F0003019B21531183216B118B2163119321739
:10030000B119B21732080800B500C030B300C030D0
:10031000B40035183314B51833163519B314B5199C
:100320003315351A3414B51AB414351B3415B51BEE
:10033000B415B416341633088316850083123408B6
:100340008316870083120034FF30B800FF30B900F5
:100350008C1EAC2914080800B90BA829B80BA629D3
:10036000FC348C1EB12914080800A000200E0F399F
:10037000BD210F302005BD210034A1000A3021022B
:1003800003183730031C3030A1072108D021003476
:100390002030D02100340D30D0210A30D02100345B
:0C03A000A2008C1CD1292208950000341A
:02400E00D230AE
:00000001FF
